S113E0007EED30BDECD6B6600881552603BDF11611
S113E010BDE0608EDFFF0E4F5FDD3ADD3FDD41BDC9
S113E020E0A37F00197F00187F001DBDE0F4BDE070
S113E030B3BDE053BDEE0F1A83000026D6DE0EDF1B
S113E0402FBDE1167D001926CA20D7DE2F6F00DF11
S113E0500E20C0BDE38C81202605BDE39520F43954
S113E060CEE0667EE10B0D0A0D0A4241534943316D
S113E070312076312E31330D0A436F70797269671E
S113E080687420313938352C313938362062790DAD
S113E0900A476F72646F6E20446F7567686D616EB6
S113E0A00D0A00CEE0A97EE10B0D0A524541445908
S113E0B00D0A00C64FCE0049BDEC58810D272B5DDB
S113E0C0272881082610C14F2720098620BDEC3B54
S113E0D08608BDEC3B5C810326067C001C7EF2298D
S113E0E0812025D4A700085A26CE860DA700CE008D
S113E0F049DF0039CEE0F920120D0A23008D00CE4D
S113E100E1088D077F001E390A0D00A6002706BD11
S113E110EC3B0820F639CEDE00DF028D33241436C2
S113E120BDE38C810D322604BDEB50397F00198D7F
S113E130672010BDE38C810D27F186019719CC006F
S113E1400020EC8D797D001927037EF1E77EEB2E0C
S113E150183C4F36361830DE00A6008D422410A637
S113E160008D3C25110D18EC0026048612200D317B
S113E170311838DF00398D072AE586017EEA4E180A
S113E180EC00050518E3000518ED00E60008C030B2
S113E1904F18E30018ED0039BDE39D4F7EE3A081E5
S113E1A0302506813922020D390C39814125068139
S113E1B05A22020D390C398DF224013920E1BDE3D4
S113E1C08C810D274F7F001ABDE346CEE224BDE3C8
S113E1D071251308A60026FBC6043A6D0026EF86B7
S113E1E002CEE3DC2004A601EE02BDE3A0810C27ED
S113E1F007810A2703BDE346AD00BDE346BDE393B3
S113E200813A2607867ABDE3A020B3810D270586CF
S113E210027EEA4E867DBDE3A0DC0283DE00CEDE14
S113E22000E7023944415441000CE3BC4C4554001E
S113E23001E3DC52454144000DEA0E524553544F6C
S113E2405245000EE3BB474F535542000FE3B2471C
S113E2504F544F0012E3B24F4E54494D450025E848
S113E260894F4E4952510026E8894F4E504143434D
S113E2700028E8A94F4E0013E83B52455455524E2E
S113E2800014E3BB49460015E8BD494E50555400FF
S113E29016E9F65052494E540003E98E3F0003E953
S113E2A08E464F520004E9264E4558540005E98134
S113E2B053544F500017E3BB454E445748001AE3EC
S113E2C0BB454E440018E3BB52454D000AE3BC5421
S113E2D0524F4E0006E3BB54524F46460007E3BB81
S113E2E05748494C450019EA41504F4B450008E74F
S113E2F0B344494D0009EA0E454550001BE7CC5094
S113E3004F525441001CE3D8504F525442001DE375
S113E310D8504F525443001EE3D8504F5254440037
S113E3201FE3D8494E425954450023EA3954494D14
S113E330450024EA49524554490027E3BB50414370
S113E34043000BEA49003CDE005FA600812026045E
S113E3505C0820F65D26023839DF00DE02C10127A1
S113E3600C867FA70008E70008DF023839C67E2044
S113E370F5DC003736A600270F8D18A100270632DA
S113E38033DD000C390820ED32330D393CDE00A6B4
S113E3900038398DF73CDE0008DF0038398D01176D
S113E3A03CDE02A70008DF028CDE8023EE86147EAA
S113E3B0EA4E86A88DEABDE15020E239DE023C86B1
S113E3C0008DDDC6028DC5810D27078DD38DC65CFA
S113E3D020F38DCC38E70039C6012004BDE51D16B5
S113E3E08DB1813D270586037EEA4E86798DB1176E
S113E3F0183C361830CEE511BDE4BD24028DA1BD14
S113E400E38C81282622BDE3958610BDE3A018A6DF
S113E41000BDE3F0BDE3938129270586047EEA4E1F
S113E4208611BDE3A07EE457BDE19F250881242722
S113E4300481222605BDE62C2009BDE7204D2603D4
S113E440BDE51D18E600C100260318A70018A100A9
S113E450270586057EEA4EBDE38C810D2740813A6F
S113E460273C81202738812C2734813B2730812980
S113E470272C18A60081012618BDE4A82518BDE4A0
S113E480B325137D001A2705BDE4B82009860020B2
S113E4900586137EEA4E4D260986067EEA4E31181D
S113E4A03839BDE3A07EE3F5CEE4D3BDE4BD250257
S113E4B0860039CEE4E620F3CEE4FB20EEBDE37122
S113E4C0250D08A60026FB0808A60026F00C39A690
S113E4D0010D392B00402D00412A00502F00515CC2
S113E4E000525E0060002E414E442E00202E4F52FA
S113E4F02E00212E454F522E0022003C3D00323E7C
S113E5003D00333C3E00353C00303E00313D00349C
S113E510002D00724000704E4F54007100183C4FA3
S113E520363636361830BDE38CBDE1AB250586079B
S113E5307EEA4E18A700BDE395BDE38CBDE1B72488
S113E5400618A701BDE395BDE5A018A703BDE5AE78
S113E5501A83FFFF260618A603BDE5E6373618A67C
S113E56003BDE3A03233BDE39D18A6038510271E27
S113E570BDE3958610BDE3A08601BDE3F0BDE39342
S113E58081292705860E7EEA4E8611BDE3A0860109
S113E59018E603C5022702860231313131183839B1
S113E5A0868436BDE38C81283226028B1039DE0A3C
S113E5B06D00272EA1002612E60118E100260BE6C5
S113E5C00218E10126048F930A39E600C5102704D6
S113E5D0C6052006C1842605C6053A20D386087ED2
S113E5E0EA4ECCFFFF39DE0E3CA7000818E600E730
S113E5F0000818E601E700088D186F00DF0E9C0C78
S113E6002304860920233233930A3736BDF29C3221
S113E610333985102704C602200681842609C602E0
S113E6206F00085A26FA3986087EEA4EBDE38CDE6E
S113E630003C81242608BDE395BDE68F2003BDE69A
S113E640613686A4BDE3A032BDE39DDC0030A300A7
S113E65017BDE3A038A600BDE3A0085A26F786013B
S113E66039183C4F36361830DE00A600BDE19F2530
S113E670048602202CA600BDE19F2409BDE17F2A67
S113E680F4860A201CDF0018EC00313118383918E0
S113E6903C4F36361830DE00A600BDE6DD250D867B
S113E6A00B7D001D27037EEAA87EEA4EA600BDE688
S113E6B0DD24D218EC0005252005251D05251A05A5
S113E6C0251718ED00E60008C030C1092302C00771
S113E6D04F18E30018ED0020D3860C20C4BDE19F41
S113E6E024013981412506814622020D390C39C69F
S113E6F00286A2BDE3A0DE023C4FBDE3A0BDE393CE
S113E700BDE3A0BDE3938122270F810D2605860D6D
S113E7107EEA4EBDE3A05C20EABDE3A038E7003901
S113E720CEE741BDE371250E08A60026FBC6043AD8
S113E7306D0026EF4F398636BDE3A0A601EE026ECA
S113E74000464449560001E7BA434852240002E710
S113E750D84142530004E7D8524E440005E7D85349
S113E760474E0006E7D85441420007E7D8414443E6
S113E7700003E7D843414C4C0008E7D85045454BCB
S113E7800009E7D8454550000AE7D8484558320003
S113E79012E7D8484558000BE7D8504F5254000CA4
S113E7A0E82154494D450011E835504143430013D5
S113E7B0E83500DE0209DF02A600183CC60137373F
S113E7C01830C602BDE7E73232183839DE0209DFF5
S113E7D002A6008D037EE3E0183CC60137C601188B
S113E7E0308D0432183839BDE3A0BDE38C8128276D
S113E7F005860E7EEA4EBDE3958610BDE3A018A6FD
S113E80000180837BDE3F0335A2707BDE9E324E1D4
S113E81020ECBDE38C812926D8BDE39586117EE3E7
S113E820A0BDE39381412405862F7EEA4E814522D3
S113E830F780418B0CBDE3A08601398601BDE3F06E
S113E840BDE346CEE24FBDE371240D8612BDE3A0C5
S113E850BDE346BDE3B22018CEE246BDE371250513
S113E860860F7EEA4E860FBDE3A0BDE346BDE3B24C
S113E870BDE346BDE9E3250139BDE34686A8BDE312
S113E880A0BDE150BDE39D20E78601BDE3F0BDE3FB
S113E89046BDE9E3250586157EEA4EBDE34686A816
S113E8A0BDE3A0BDE1507EE39D8D0220DC8601BD69
S113E8B0E3F0BDE346BDE9E324DC7EE3467C001AD5
S113E8C08601BDE3F0BDE346CEE91CBDE371250539
S113E8D086107EEA4E8638BDE3A0BDE346BDE38CD8
S113E8E0BDE19F242786A8BDE3A0BDE150BDE39D03
S113E8F0BDE346CEE921BDE3712501398639BDE387
S113E900A0BDE346BDE38CBDE19F250586127EEAEA
S113E9104E86A8BDE3A0BDE1507EE39D5448454E1C
S113E92000454C534500BDE51D8101270586037E46
S113E930EA4EBDE393813D26F48679BDE3A08601CA
S113E940BDE3F0BDE346CEE979BDE371250586114B
S113E9507EEA4E8637BDE3A0BDE3468601BDE3F003
S113E960BDE346CEE97CBDE371250139863ABDE3BA
S113E970A0BDE34686017EE3F0544F005354455056
S113E98000BDE51D8101270586027EEA4E39BDE3FF
S113E9908C8123260D8678BDE3A0BDE395BDE346B7
S113E9A0201BBDE346BDE38C810D2704813A26017B
S113E9B039BDE38C81222605BDE6EF20058601BD25
S113E9C0E3F0BDE346BDE38C810D27E4813A27E003
S113E9D08D1125CE813B270586167EEA4E867B8DDA
S113E9E00D20BFBDE38C812C27020C39867CBDE34E
S113E9F0A0BDE3950D398D21BDE346BDE38C812295
S113EA00260CBDE6EF8DDC250586157EEA4EBDE5B8
S113EA101DBDE3468DCD25F639BDE38C8123270149
S113EA20398678BDE3A0BDE395BDE3468601BDE329
S113EA30F0BDE3468DAD24D1398DDEBDE3467EE5E0
S113EA401D7C001A86007EE3F0C6017EE3E0971881
S113EA50BDE0FDCE0049A600810D2706BDEC3B08B4
S113EA6020F4BDE0FFDE0009098C0049230FDF001C
S113EA70CE0049862ABDEC3B089C0026F8CEEA9BD2
S113EA80BDE10BBDE0FF8D078601971C7EE04BCEF8
S113EA90EA9FBDE10BD6184F7EEACE5E5E5E00456E
S113EAA052524F52202320009718BDEA8FCEEAC25B
S113EAB0BDE10BDC29BDEACEBDE0FF20CB425245CF
S113EAC0414B20494E204C494E45202320001A83B7
S113EAD00000260586307EEC3B183C3736CC2710E8
S113EAE037365F37183018EC032A0D4353C300013F
S113EAF018ED03862DBDEC3B18EC03CDEE01021896
S113EB00ED038F1A8300002605186D00270B178B61
S113EB1030C60118E700BDEC3B18EC01CE000A0238
S113EB20CDEF0126D3C605183A18351838398601B1
S113EB30971CFCDE001A93102309BDEC0BFCDE00CD
S113EB40DD10398D50EC001AB3DE0026677EEC210F
S113EB50373618301A931023078601971C3233393D
S113EB608D33EC00CDA30026F0E6028D0DDC10CD34
S113EB70A30026E58D2EDD1020DF183C3C18381844
S113EB803A189C06240A18A600A70008180820F1C1
S113EB90DF06183839DE041AA300230737E6023AE1
S113EBA03320F439DE049C062709EC0037E6023AE8
S113EBB03320F339F6DE023C8D0338203B183C3C0D
S113EBC0DE063C3A3C183018EC001A9308230B86F6
S113EBD0097EEA4E383838183839DD0618EC02CD8B
S113EBE0A30425F0CDEE02A60009CDEF02CDEE0080
S113EBF0A70009CDEF0020E4F6DE0218CEDE0018EF
S113EC00A6001808A700085A26F539DE06F6DE0223
S113EC103A9C0822078FDE06DD0620DC86097EEAA0
S113EC204EE602F0DE02260220CE2A08503CBDEB5E
S113EC30BD3820C43CBDEB7A3820BD7C001E373C77
S113EC40CE00B4D637583AEE0026087F0037863116
S113EC507EEAA8AD00383339373CCE00A420E48DD9
S113EC600D36B69800850227F932B7980139B6985F
S113EC7000850127F9B698013936B6980085013226
S113EC8039B6102E842027F9B6102F3936B6102E37
S113EC90858027F932B7102F3936B6102E852032E9
S113ECA0398632B7102B7F102C860CB7102D8611A5
S113ECB0974386139744398613B798008656B798B6
S113ECC000398DD5270E368DB8914426068DB29124
S113ECD04326FA3220B6CED000B66008815526030A
S113ECE0CEC000DF0ADF0E6F00088CDDFF26F8DFE0
S113ECF00CB660088155260FFC6000DD04FC600240
S113ED00DD06BDF34C2011CEC000DF04DF066F002A
S113ED10088CCFFF26F8DF08CC0000DD10DD29BD0C
S113ED20F2407F001B8601971CB7A0007F00373993
S113ED308693B710398603B710248EDFFFCE00C444
S113ED4018CEEDC2C614867EA700081AEF00080884
S113ED505A26F5979E97A1CCEC79DD9FCCEC6EDD1D
S113ED60A2CE00F7CCED30ED01ED04ED07CE00A40A
S113ED70C6206F00085A26FACEEC5FDFA4CEEC6101
S113ED80DFB4CEEC81DFA6CEECC2DFB6CEEDC0DFC1
S113ED90E08603973C7F00387F00398680B71022D5
S113EDA08D21CEEDFEDFEFCEEE04DFCBDFCE4F5F65
S113EDB0DD3DDD3FDD410EBDECB7BDECA17EE003E2
S113EDC08D013BFC1016C3F424FD10168680B71089
S113EDD0237A003C26278602973CDC38C30001DDF9
S113EDE038DC3A27181A9338261318DE3D31317C63
S113EDF00019DC29DD45DC2BDD477EF3E63918DE1E
S113EE003F26EC3B8630B7102518DE4126E13BBD9A
S113EE10E38C810D2604CC000039CEEE38BDE371BD
S113EE20250E08A60026FB0808086D0026EF20E63C
S113EE30EE01AD00CC0001394C49535400EE85522B
S113EE40554E00F1164E455700F286434F4E54007E
S113EE50F271434C45415200F299455341564500E5
S113EE60F2B0454C4F414400F32E4C4C49535400EE
S113EE70F36F4155544F535400F37A4E4F41555458
S113EE804F00F38300BDE0FDDC041A93062601392C
S113EE90BDE053BDE38CBDE19F2427BDE150DD12ED
S113EEA0BDE38C812D270ADC12DD141A9310232173
S113EEB039BDE395BDE1501A93102302DC10DD1433
S113EEC0200F810D270139DE04EC00DD12DC10DD9A
S113EED014DC121A9314230139DC12BDEB95DF0202
S113EEE0DC14BDEB95EC001A93142603E6023ADF1A
S113EEF014DC021A9314260139DE02EC0008080817
S113EF00DF02BDEACEDE02A600817D270D4D2B0572
S113EF10BDEF9820F0BDEF2420EBBDE0FFDE02083A
S113EF20DF0220CDDE02A60084EFCEEF42A100274F
S113EF300C0808086D0026F586087EEA4EEE01AD41
S113EF40003984EF4FA2EF84A8EF8BA4EF7D00DE9D
S113EF500208EC00D30A0808DF028FA601BDEC3BCF
S113EF60A6022703BDEC3B39DC02C300068FE60092
S113EF7008A600BDEC3B085A26F7DF0239DC02C3C1
S113EF80000320E9DC02C3000120E2DE0208EC00F9
S113EF900808DF02BDEACE39DE02A60008DF0281DE
S113EFA07F26037EEFDC810A26037EEFF4810C26A4
S113EFB0037EEFEC8136260CDE02A60008DF02CECB
S113EFC0F0C82003CEF00DA100270C0808086D003E
S113EFD026F586087EEA4EEE017EE10BDE02E600AF
S113EFE008DF028620BDEC3B5A26FA39CEE224BD66
S113EFF0E10B2006CEE2C8BDE10BDE0208A60081CB
S113F0000D260408DF0239BDEC3B0820F001E22C98
S113F0100DE2330EE23B0FE24612E24F13E27414A8
S113F020E27A15E28438E91C39E92116E28A03E21E
S113F0309304E2A105E2A817E2B018E2C106E2CF08
S113F04007E2D719E2E01AE2B83AE97C37E9797CB9
S113F050F1067BF1047AF10202F10108E2E979E5B3
S113F0600D10F10811F10A20E4E621E4ED22E4F3A5
S113F07030E50731E50A32E4FB33E4FF34E50D35CE
S113F080E50340E4D341E4D650E4D951E4DC52E44E
S113F090DF71E51760E4E272E5117EF10C09E2F13B
S113F0A01BE2F81CE2FF1DE3081EE3111FE31A78BC
S113F0B0F11423E32324E32D25E25726E26127E319
S113F0C0350BE33D28E26A0001E74102E74903E723
S113F0D06D04E75105E75806E75F07E76608E7743C
S113F0E009E77C0AE2F80BE7930CE2FF0DE3080E54
S113F0F0E3110FE31A10F10E11E32D12E78B13E362
S113F1003D003A003B002C00280029002000504F0D
S113F110525445002300BDE0FDBDF2408601971D19
S113F12018DE04189C0626013918EC00DD297D0040
S113F1301B2712865BBDEC3BDC29BDEACE865DBD98
S113F140EC3BBDE0FF183C18E602183A18DF2B1818
S113F15038C603183A7A001A2603BDF2198D281806
S113F160E60018088D215A58CEF1973AEE00AD000A
S113F1708D1518A600817D260A1808189C0626A954
S113F1807EF46B180820CE18A6002B0A817E270473
S113F19025041808180839F38DF38DF5AEF717F721
S113F1A06FF5A5F5AAF55EF6A6F387F9C3F387F81C
S113F1B08BF8AEF41A00000000F3D7F4FBF447F820
S113F1C0E8F7AFF45BF46BF48FF4D5F911F57EF541
S113F1D096F59BF5A0000000000000F9A6F9B8F927
S113F1E0D7F9EEFA0CFA2EBDE0FD18CEDE0018ECCD
S113F1F000DD29C603183A8D8E18E60018088D879D
S113F2005A58CEF1973AEE00AD00BDF18718A6002A
S113F210817D260139180820DE860A971A9D9E26CC
S113F22001399DA1810327013918DF31BDE0FFCEEB
S113F230EABDBDE10BDC29BDEACEBDE0FF7EE013F3
S113F240BDF299CEDEDADF1FCEDE9EDF21CEDF2ACD
S113F250DF23CEDF3ADF25CEDF4ADF27DE0E08DFED
S113F2602D7F001E860A971A7F001CCE0000DF3314
S113F27039BDE0FD7D001C260618DE317EF15D8679
S113F2802597187EEA8FB660088155260886FFB751
S113F2906008BDF99DBDECD639BDF243DE0AA60077
S113F2A02708080808BDE61220F4DE0E08DF2D3911
S113F2B0DE049C06260139CC600BB76000BDF99DC5
S113F2C0F76001BDF99D188FA6000818A700BDF9C5
S113F2D09D18089C0626F1188FB76002BDF99DF7AA
S113F2E06003BDF99DDC10B76009BDF99DF7600AA4
S113F2F0BDF99DDE0A9C0E2731FC6002B76004BD97
S113F300F99DF76005BDF99D188FA6000818A700A0
S113F310BDF99D18089C0E23F11809188FB76006D3
S113F320BDF99DF76007BDF99D394F5F20EFFE6081
S113F3300026013918DE04A60018A700081808BC26
S113F340600226F318DF06FC6009DD10FE60062665
S113F35005DE0ADF0E39FE600418DE0AA60018A7CF
S113F36000081808BC600623F3180918DF0E398654
S113F370019737BDEE857F0037398655B76008BDE4
S113F380F99D3986FF20F518E600183A3918A600C9
S113F3908D0E37361808BDFA85BDFB2D38ED0039C2
S113F3A018A6008502261D8510260F18EC01D30A25
S113F3B0C3000337C603183A3339BDFB043C300598
S113F3C0E3003839851027E3BDFB043C37363005AC
S113F3D0E30031313020E97D00192704DC06DD2B00
S113F3E0DE2B9C062604DE042007EC00CDA30122BC
S113F3F0F5EC00CDA30127102505861B7EEAA8E6BF
S113F400023A9C0627F420E98F188F7D00192706FD
S113F4107F00197EF17B313120F9183C7D001927DA
S113F4200718DE0618092004C603183ABDF187DE62
S113F4302709098CDF3A2405861C7EEAA8DF271AEF
S113F440EF0018387EF3D7DE278CDF4A2605861DA9
S113F4507EEAA81AEE000808DF2739CEF47ABDE167
S113F4600BDC29BDEACE18DF312007BDE0FF8601A1
S113F470971CCC0000DD297EE0130A0D53544F5035
S113F480504544204154204C494E4520232000DE61
S113F4902509098CDF2A2405861E7EEAA8DF251AA1
S113F4A0EF00C6013718DE2B260139183C189C06DC
S113F4B027B9DE2BE6023ADF2BC603183ABDF187E3
S113F4C018A600183833811926015C811A26D55AEA
S113F4D026D27EF416DE258CDF3A2605861F7EEAC8
S113F4E0A8183C1AEE00BDFA85BDFB2D260A183873
S113F4F0DE250808DF252002313139BDFA85BDF14A
S113F5008718A600361808BDF187DE1FEC002A070D
S113F510260586207EEAA8EC008300012717ED006B
S113F520C603183ABDF18718A600817D27E41808A0
S113F530BDF18720E2BDFB2D32811226037EF3D775
S113F540183CC603183ABDF18718A600817D270B25
S113F550817A27071808BDF18720E77EF42C180864
S113F560BDF187BDFA85BDF1871808BDF187BDFAE5
S113F570851808BDFB2D8FBDFB2D8FE70039CE10FC
S113F580003C1808BDFA85BDFB2D4D2705862E7E4F
S113F590EAA838E70039CE100420E6CE100320E1B3
S113F5A0CE100820DC86FF971B397F001B39BDF77E
S113F5B0ED18A600817D2704817A2607BDE0FF7F30
S113F5C000373981A22616183CC60218EB01183AF6
S113F5D03808E600C0020808BDF8672039813626DD
S113F5E01E18A60181072605BDF65320298102268F
S113F5F005BDF6682020810B2605BDF67C20178109
S113F600122605BDF674200EBDFA85BDFB2DBDEA9C
S113F610CE8620BDEC3BBDF18718A600817C27086F
S113F620817B2628180820131808D61EC40750CB3F
S113F6300827088620BDEC3B5A26FABDF18718A698
S113F64000817D270A817A27067EF5C3BDE0FF7F0E
S113F6500037398D432705862A7EEAA8D11E230761
S113F6608620BDEC3B20F5398D2E2704862B20E91E
S113F670177EEC3B8D222708863220DD8D1A8D0102
S113F68017368D0332200444444444840F8B308164
S113F6903923028B077EEC3BC603183ABDFA851862
S113F6A008BDFB2D4D3918A6008510260586217E40
S113F6B0EAA818EC01D30A8FEC032704862220EF72
S113F6C03CC604183ABDFA85180838DC2DED03C38E
S113F6D00002DD2DBDFB2D2A04862720183CEE03F5
S113F6E0ED00C300013805D32D1A932D23051A9379
S113F6F00C230586097EEAA8DD2DEE0308086F00B9
S113F700089C2D26F9BDF18718A600817D270718CE
S113F71008BDF187209039DC2383000A1A83DEDADE
S113F720240586237EEAA8DD23183CBDF3A01838FF
S113F730DE23ED00DC29ED08BDF38DBDF18718084B
S113F740BDF187BDFA85BDFB2DDE23ED04CC0001A0
S113F750ED02BDF18718A600813A27041AEF063995
S113F7601808BDF187BDFA85BDFB2DDE2320E1BD60
S113F770F3A0DE231AA300270586247EEAA8183CFA
S113F7801AEE0018EC00E30218ED006D022B111ABA
S113F790A3042F1118388FC3000ADD23BDF1873964
S113F7A01AA3042DEF18381AEE06EC08DD29398D5A
S113F7B03C18A60081A2261B183CC60218EB0118AF
S113F7C03A3808E600C0020808BDF8671808BDF119
S113F7D0872003BDE0FFCEF7EABDE10BBDE0B38DAA
S113F7E03B25F0BDE0FF7F0037393F200018A6001D
S113F7F081782701391808BDF187BDFA85BDFB2D35
S113F8002A0586307EEAA81A83000722F5D737BD79
S113F810F187817D27051808BDF18739BDE0538143
S113F8200D26020D398D13BDF18718A600817D26A2
S113F830020C391808BDF18720E281242608BDE3B3
S113F84095BDE68F2003BDF8743736BDE053812C97
S113F8502709810D270886157EEAA8BDE395BDF327
S113F860A08F3233ED00395D2709A60008BDEC3BBB
S113F8705A26F739BDE38C812D260CBDE395BDE6F0
S113F880614353C3000139BDE66139DE3326048D7B
S113F8901DDE33DF00BDF81C2505DE00DF3339181B
S113F8A03C18DE00180818088D3A183820DD183C7A
S113F8B018DE04183C18E602183A18DF331838C664
S113F8C003183ABDF18718A600810C270D18DE3302
S113F8D0189C0626DE86267EEAA81808180818DF73
S113F8E033183839183C20E8BDFA85BDF18718086B
S113F8F0BDF187BDFB2D27037EF3D7C603183ABDA0
S113F900F18718A600813926071808BDF18720E879
S113F910391808BDF187BDFA8518081808BDFA859D
S113F920183C18DE1F18EC022B061A8300FF23056F
S113F93086287EEAA805C3B6008FA60081FF2702A9
S113F9408D1D08A60081FF27028D1418A6018D2B9A
S113F9500918A6008D251838BDFB2DBDFB2D39C611
S113F96016F7103BA70007360FC617F7103B8D2D6F
S113F970C616F7103B32067F103B39C602F7103B20
S113F980A7003607360FC603F7103B8D10C602F7E3
S113F990103B32067F103B32A10026DF393CCE0DEE
S113F9A0020926FD3839BDF7EDBDF3A08FBDEC5833
S113F9B0164FED007F0037391808BDFA85BDFB2DC1
S113F9C0DD38391808BDFA85BDFB2D4D2705863570
S113F9D07EEAA8F71027398D4ABDFA85BDFB2DDDD7
S113F9E03ABDF1871808BDF18718DF3D20198D3322
S113F9F0BDFA85BDF1871808BDF187BDFB2D26042E
S113FA00DD3F200318DF3FC603183A398D150785FB
S113FA1010260586347EEAA8DC45DD29DC47DD2B8B
S113FA2031313B7D0019270586337EEAA8398DF3F1
S113FA30BDFA85BDF1871808BDF187BDFA85BDF112
S113FA40871808BDF18707360F18DF41BDFB2D1A53
S113FA50830001230586367EEAA886105D270148C7
S113FA60B71024BDFB2D26077F1026DD41200F1A79
S113FA7083000422E0CB0358585858F71026320666
S113FA80C603183A398610BDFB8F18A600811026CC
S113FA900818088DF0180820F14D2A048D1220EA68
S113FAA0BDFB3CBDFB7F2401391808BDFB8F20DA68
S113FAB08184260E18EC01D30A8FC603183AEC038E
S113FAC0202D81A4260DCDEE01C60418EB03183AAF
S113FAD08F201C819426138D2B183C3C051830185C
S113FAE0E3003818388FEC00200586087EEAA8DE8B
S113FAF01F09098CDE9E2407861797187EEAA8DF63
S113FB001FED003918EC01D30A8FEE032605861881
S113FB107EEAA8C604183A3CBDFA85180838BDFB2D
S113FB202D1AA3002304861920E60808393CDE1F99
S113FB30EC000808DF1F381A8300003981362701DA
S113FB403918A6014AC603183A1658CEFB593AEE9C
S113FB5000AD00180818A60039FD95FE14FDBAFD85
S113FB603DFDEDFD4EFE14FD60FD6BFD7AFE14FEC1
S113FB7023FE2EFE33FE38FE3DFE19FE14FE1D81CB
S113FB80112708817A24020C3986118D020D39DE81
S113FB9021098CDE80260586177EEAA8DF21A700CE
S113FBA0DE21A60081102719E601C4F084F0112299
S113FBB010A601E600C1112609811026050808DFF8
S113FBC02139E70108DF218D0220D58170250780C6
S113FBD070CEFC19203C816025078060CEFC1F207C
S113FBE031815025078050CEFC21202681402507F5
S113FBF08040CEFC27201B813025078030CEFC2B93
S113FC002010812025078020CEFC37200586087E21
S113FC10EAA816583AEE006E00FCF5FCF6FCFFFD6F
S113FC203CFCC7FC75FCC1FC5FFC68FD07FD12FDD4
S113FC3018FD1EFD24FD2AFC54FC49FC3DBDFB2D92
S113FC40DE1FA800E801ED0039BDFB2DDE1FAA0070
S113FC50EA0120F2BDFB2DDE1FA400E40120E7BD74
S113FC60FB2DDE1FE30020DEDE1FEC02A3000808EC
S113FC70ED00DF1F398D08BDFB2DDE1FED0039DEE1
S113FC801FA600A80236EC002605861A7EEAA82ADA
S113FC9003BDFCFF6D022A09EC024353C30001EDCE
S113FCA002EC00EE028F023CDE1FED023233ED0067
S113FCB0324D2A0CBDFCFFEC024353C30001ED029C
S113FCC0398DBCBDFB2D39183CDE1FA601E6033D72
S113FCD037361830A601E6023D18EB0018E700A6F7
S113FCE000E6033D18EB0018E70008083233ED0086
S113FCF0DF1F18383939DE1FEC004353ED00398D0E
S113FD00F5C30001ED00398D272C026C030808DFD0
S113FD101F398D1C2FF720F38D162EF120ED8D1039
S113FD202DEB20E78D0A26E520E18D0427DF20DB7B
S113FD30DE1FEC026F026F031AA3003939BDFA8586
S113FD40DE1FEC002A054353C30001ED0039BDFA60
S113FD5085DE1FEC0027F4CC00016D002AED20E6BF
S113FD60BDFA85DE1FEE00AD00200ABDFA85DE1F58
S113FD70EE00E6004FDE1FED0039BDFA85DE1FEC14
S113FD80001A8300FF230586287EEAA805C3B6006F
S113FD908FEC0020E0BDFA85BDF1871808BDF1871E
S113FDA0BDFA85DE1FEC02EE00032804862C20D960
S113FDB08FDE1F0808ED00DF1F39BDFA85DE1FEC5A
S113FDC0002B061A8300072304862D20E1F7103048
S113FDD07D10302AFB4FF61031FB10328900FB10E6
S113FDE0338900FB103489000404ED0039BDFA8521
S113FDF0DE1FEC00270B2B04DC352014FC100EDD79
S113FE0035DC35581BD6360505D335C33619DD35F3
S113FE1004ED003986297EEAA8DC38200AF610278A
S113FE204F2004F610004F180918097EFAEFF61057
S113FE300420F3F6100320EEF6100820E9F6100A69
S113FE4020E4FFFFFFFFFFFFFFFFFFFFFFFFFFFFB8
S113FE50FFFFFFFFFFFFFFFFFFFFFFFFFFFFFFFFAE
S113FE60FFFFFFFFFFFFFFFFFFFFFFFFFFFFFFFF9E
S113FE70FFFFFFFFFFFFFFFFFFFFFFFFFFFFFFFF8E
S113FE80FFFFFFFFFFFFFFFFFFFFFFFFFFFFFFFF7E
S113FE90FFFFFFFFFFFFFFFFFFFFFFFFFFFFFFFF6E
S113FEA0FFFFFFFFFFFFFFFFFFFFFFFFFFFFFFFF5E
S113FEB0FFFFFFFFFFFFFFFFFFFFFFFFFFFFFFFF4E
S113FEC0FFFFFFFFFFFFFFFFFFFFFFFFFFFFFFFF3E
S113FED0FFFFFFFFFFFFFFFFFFFFFFFFFFFFFFFF2E
S113FEE0FFFFFFFFFFFFFFFFFFFFFFFFFFFFFFFF1E
S113FEF0FFFFFFFFFFFFFFFFFFFFFFFFFFFFFFFF0E
S113FF00FFFFFFFFFFFFFFFFFFFFFFFFFFFFFFFFFD
S113FF10FFFFFFFFFFFFFFFFFFFFFFFFFFFFFFFFED
S113FF20FFFFFFFFFFFFFFFFFFFFFFFFFFFFFFFFDD
S113FF30FFFFFFFFFFFFFFFFFFFFFFFFFFFFFFFFCD
S113FF40FFFFFFFFFFFFFFFFFFFFFFFFFFFFFFFFBD
S113FF50FFFFFFFFFFFFFFFFFFFFFFFFFFFFFFFFAD
S113FF60FFFFFFFFFFFFFFFFFFFFFFFFFFFFFFFF9D
S113FF70FFFFFFFFFFFFFFFFFFFFFFFFFFFFFFFF8D
S113FF80FFFFFFFFFFFFFFFFFFFFFFFFFFFFFFFF7D
S113FF90FFFFFFFFFFFFFFFFFFFFFFFFFFFFFFFF6D
S113FFA0FFFFFFFFFFFFFFFFFFFFFFFFFFFFFFFF5D
S113FFB0FFFFFFFFFFFFFFFFFFFFFFFFFFFFFFFF4D
S113FFC0FFFFFFFFFFFFFFFFFFFFFFFFFFFFFFFF3D
S113FFD0FFFFFFFFFFFF00C400C700CA00CD00D031
S113FFE000D300D600D900DC00DF00E200E500E821
S113FFF000EB00EE00F100F400F700FA00FDED3034
S9030000FC
